:100000008A110A120528000009000730990083169A
:100010000510851005110512851283120510851033
:10002000051105128512EE30B1000230B2007830B1
:10003000B300B4013308B5003408B6003308A60095
:100040003408A7000430A200A3017B22B7002508D2
:10005000B8003308A6003408A7001430A200A3019A
:100060007B22B9002508BA000530B0008501BC30FC
:10007000A0000230A1009122AC012C08643C031CBA
:10008000552805148516851005124630A000A101DB
:10009000912205108512851405164630A000A10195
:1000A00091220130AC07031C3D281F3083058501D8
:1000B000BC30A0000230A1009122DF202C30AE0025
:1000C0000130AF00AC012C081E3C031C8528051430
:1000D0008516851005122E08A0002F08A100912278
:1000E00005108512851405162E08A0002F08A10002
:1000F00091220A302E02AE000030031C013E2F0276
:10010000AF000130AC07031C63281F308305850155
:10011000AC012C080A3C031CA32805148516851481
:100120000516F430A0000130A100912285100512BF
:10013000051085122C30A0000130A1009122013061
:10014000AC07031C89281F3083058501AC012C08EE
:10015000643C031CBF280514851685100512463023
:10016000A000A101912205108512851405164630C4
:10017000A000A10191220130AC07031CA7281F3069
:10018000830585018501F430A0000130A100912292
:10019000FF308500D030A0000730A10091228501FA
:1001A000F430A0000130A1009122FF308500D03052
:1001B000A0000730A100912285013628DE28F43006
:1001C000A0000130A10091226321EB216321EB21EA
:1001D000632106223C21EB215F21EB21A521EB21AC
:1001E0002021EB21472106220F21EB216321EB2166
:1001F0002021EB213C21EB213C21EB210F21EB21A4
:100200004421EB212021EB211C21EB210F2106228F
:1002100085019030A0000130A10091220800352214
:100220004C2208004C2235223522352208004C226F
:1002300035224C22352208004C2235223522080076
:1002400035220800352235224C22352208004C2266
:100250004C2235220800352235223522352208006D
:1002600035223522080035224C224C224C2208002F
:100270004C2235224C22080035224C2235223522D0
:1002800008004C224C2208004C22352208004C2247
:100290004C224C22080035224C224C2235220800E8
:1002A0004C224C2235224C22080035224C22352289
:1002B000080035223522352208004C22080035225C
:1002C00035224C2208003522352235224C220800E6
:1002D00035224C224C2208004C22352235224C2259
:1002E00008004C2235224C224C2208004C224C2281
:1002F0003522352208004C224C224C224C224C2222
:10030000080035224C224C224C224C220800352277
:1003100035224C224C224C2208003522352235222F
:100320004C224C22080035223522352235224C221F
:1003300008003522352235223522352208004C228C
:10034000352235223522352208004C224C22352216
:100350003522352208004C224C224C2235223522EF
:1003600008004C224C224C224C2235220800352217
:100370004C2235224C2235224C2208004C224C22A1
:10038000352235224C224C220800352235224C22BF
:100390004C223522352208004C22352235224C22AF
:1003A000352208004C223522352235224C22080005
:1003B0004C2235223522352235224C2208000510E8
:1003C0003308A0003408A10091223308A0003408AB
:1003D000A1009122080005103308A0003408A100F4
:1003E00091223308A0003408A10091223308A00014
:1003F0003408A10091223308A0003408A100912202
:100400003308A0003408A100912208000510330829
:10041000A0003408A10091223308A0003408A100F4
:1004200091223308A0003408A10091223308A000D3
:100430003408A10091223308A0003408A1009122C1
:100440003308A0003408A10091223308A00034082A
:10045000A10091223308A0003408A10091223308A2
:10046000A0003408A1009122080005148514051687
:100470008516053084000430AA003108A000320837
:10048000A1003508A2003608A300CC220510851073
:1004900005128512DF21080005148514051685163E
:1004A000053084000430AA003108A0003208A10001
:1004B0003708A2003808A300CC22051085100512C9
:1004C0008512DF21080005148514051685160530F0
:1004D00084000430AA003108A0003208A1003908C5
:1004E000A2003A08A300CC2205108510051285123F
:1004F000DF2108007A2A1030A800A101A001A70C72
:10050000A60C031C892A2208A00723080318230F1E
:10051000A107A10CA00CA50CA40CA80B7F2A2408F1
:100520000800A00803199C2AA322A00300000000D1
:10053000000000000000912AA10803190800A3226E
:10054000A103A003912A0C30A500A50BA52A000049
:1005500000001230A200A20BB22AB422B422000082
:1005600000000800B422AB2A0D30A400A40BB62A68
:10057000000008001030A8020001031C013EA9027F
:10058000031C0800C32A0A30A8020001031C013E14
:10059000A902031C0800C32A2A0880042008A80016
:1005A0002108A900BA220130A202031CA3032A09D0
:1005B00080052008A8002108A900BA22A208031D6E
:0A05C000CC2AA308031DCC2A080072
:02400E00C431BB
:00000001FF
